:020000040000FA
:020000000528D1
:080008009829831203138501FE
:10001000831606309F00CF30850007309C00831682
:100020000030850086000F308700FF3088001730D1
:1000300089008C178312C0308B00C00185018601B6
:10004000870188018901712125211F216821222131
:1000500068215621C2205621CD201F215921380860
:100060006E21492137086E21492136086E21492128
:1000700035086E21492134086E2149212E3049214D
:1000800033086E21492132086E21492131086E2141
:100090004921203049213A086E21492139086E2131
:1000A00049213F086E21C7003F30C7020319D820FD
:1000B000222102305F2130086E2149213F08C6000D
:1000C0001630C602031D6B213F086E2149214B30BB
:1000D0004921683049217A304921203049210930AD
:1000E0005F213E086E2149212E3049213D086E21B5
:1000F00049213C086E2149214B3049216830492172
:100100007A3049212D28820746347234653471349F
:10011000753465346E346334793420344334683450
:1001200061346E3400348207423461346E34643496
:10013000773469346434743468342034203442347D
:10014000463430340034820753345334423420343C
:100150004F347034653472346134743469347634B5
:100160006534003482074634693478346534643445
:100170002034423457342034263420344234463438
:100180004F340034C0011F2140088320003A031976
:10019000CC284921C00AC3280034C00122214008CC
:1001A0009320003A0319D7284921C00ACE280034E9
:1001B000222168215621C0014008A320003A0319DA
:1001C000E4284921C00ADC28C00159214008B22096
:1001D000003A0319EE284921C00AE62873211F219D
:1001E000592138086E21492137086E2149213608E6
:1001F0006E21492135086E21492134086E2149219B
:100200002E30492133086E21492132086E214921BF
:1002100031086E214921203049213A086E214921B7
:1002200039086E2149213F086E21C8003F30C802BD
:100230000319EE28222168215621CD2000340030F8
:10024000C50000340130C50000341F2120303C219E
:1002500028303C2106303C210C303C2168217B2198
:10026000222120303C2128303C2106303C210C301A
:100270003C2168217B210034C400440E0F398600E4
:1002800085108A2144080F39860085108A2179213A
:100290000034C400440E0F39860085148A214408B6
:1002A0000F39860085148A217B21003480303C215F
:1002B0000034C0303C210034803E3C210034C03E3C
:1002C0003C2100340D303C2100340C303C21003402
:1002D00001303C2100342E30492108000F39303ED6
:1002E000080064307E2950307E2932307E29143057
:1002F0007E290A307E2905307E290130C100C730B1
:10030000C2000530C300C20B8629C30B8329C10B71
:100310007F290034451C9021451C00349421003471
:100320000515000005110034851500008511003405
:10033000A200030E8301A00007080F39303E84009D
:10034000080880008C13200E8300A20E220E0900E4
:02400E00723FFF
:00000001FF
